:0D055B000B163F065B4F666D7D077F6F3905
:10044C00E4FDFCC293EF7004790D8002790FE4FB9C
:10045C00C292E930E304D2918002C291D292E92592
:10046C00E0F90BBB04EAD291C292E4FBED25E0FD6E
:10047C00EC33FCD292C292309105430501800353B8
:0E048C0005FE0BBB0CE6D293EC540FFEEDFF09
:01049A00223F
:1004E000E4FFE4FE74212FF8E6FD30E704D29580A6
:1004F00002C295D29674212FF8ED25E0F6C2960E31
:0B050000BE08E10FBF04DBD294C294E0
:01050B0022CD
:1003F00012050CE4FBFA7920784112010612024A38
:100400008E138F147C007D641202CB74162FF8E6D5
:10041000F524AE13AF147C007D641202CB8C138DD7
:1004200014AE13AF147C007D0A1202CB74162FF8A1
:10043000E6F523432380AE13AF147C007D0A12023D
:0C044000CB74162DF8E6F5228520212251
:100546000512D3E5126480948A4009E4F512120379
:05055600F01204E02298
:10049B00850E10850F11850C0E850D0F850A0C85A9
:1004AB000B0D85080A85090BE4FF12044C8E088F8F
:1004BB0009E509250BCFE508350ACF250DCF350CFE
:1004CB00CF250FCF350ECF2511CF3510FE7C007DFC
:0504DB000512032022C0
:10050C0012049BAC06AD07EC1202117B017A4D79FB
:10051C0004783D1201067BB67AF3797178C112002A
:02052C00152296
:03000B00020003ED
:06000300438CDC05153200
:10052E00D2AFD2A9438901D28CE4F515E51560FC52
:08053E00E4F51512054680F4F6
:10000E000202B6E86480F8E933E83360110460F068
:10001E00ED33EC337009E8FCE9FDEAFEEBFF220458
:10002E0060DED3EB9FEA9EE99DE8C2E78CF0C2F753
:10003E0095F0400CE8CCF8E9CDF9EACEFAEBCFFB1F
:10004E0012028185D0F05804700320D5B3E80470F5
:10005E00075002B2D50202C092D5EC0460F7E4CC90
:10006E00C0E0C398F8603B94186008400DD0E0FBE8
:10007E00020298E4FBFAC9FC8028E830E406E4C9E1
:10008E00FBE4CAFCE830E305E4C9CACBFCE854073C
:10009E006010F8C3E913F9EA13FAEB13FBEC13FC47
:1000AE00D8F130F52FC3E49CFCEF9BFFEE9AFEEDEA
:1000BE0099FDD0E0FBEF4E4D4C701222DB03020295
:1000CE00BDEC2CFCEF33FFEE33FEED33FDED30E7F0
:1000DE00EB020298EF2BFFEE3AFEED39FDD0E0FB7E
:1000EE0050130BBB00030202C0ED13FDEE13FEEF27
:0800FE0013FFEC13FC02029851
:10010600EC4D6011E8497017ED33EC3304600DE4F3
:10011600FCFFFEFD22E933E8330470F80202B61252
:10012600028158046009E4CC248150062850090253
:1001360002C02840030202BDC0E0EB4A7044B98009
:1001460006D0E0FB0202ACEF4E701CBD8008EBFF50
:10015600EAFEE9FD80EBE98DF0A4FEE5F00201EF91
:10016600E9CDF9EAFEEBFFEF89F0A4FCE5F0CE89D4
:10017600F0A42EFFE435F0CD89F0A42DFEE435F091
:100186008067EF4E7005BD80D780C3EF8BF0A4ACBF
:10019600F0EE8BF0A42CFCE435F0F8EF8AF0A42CFA
:1001A600E5F038FCE433CB8DF0A42CFCE5F03BF80D
:1001B600EE8AF0A42CFCE5F038F8E433CF89F0A4FD
:1001C6002CFCE5F038CF3400CE89F0A42FFFE5F003
:1001D6003EFEE433C98DF0A42EFEE5F039CD8AF05B
:1001E600A42FFFE5F03EFEE43DFD33D0E0FB5007D3
:1001F6000BBB000F0202C0EC2CFCEF33FFEE33FE0C
:06020600ED33FD02029839
:10020C0075F020800E75F010800575F0087D007E6D
:10021C00007F003392D530D503120356EC334010D7
:10022C00EF33FFEE33FEED33FDEC33FCD5F0ED2276
:0E023C00E5F0247EA2D513CC92E7CDCEFF22B2
:10024A00EDD2E7CD33EC3392D524814006E4FFFEAC
:10025A00FDFC22FCE4CFCECDCC24E0501174FF800B
:10026A00EDC3CC13CCCD13CDCE13CECF13CF0470A8
:07027A00F030D5DE0203564F
:10028100E9D2E7C933E833F892D5EDD2E7CD33ECC3
:0702910033FC5002B2D5223C
:10029800EC30E7100FBF000C0EBE00080DBD0004C7
:1002A8000BEB6014A2D5EB13FCED92E7FD2274FF73
:1002B800FCFDFEFF22E480F8A2D574FF13FC7D80CC
:0302C800E480EFE0
:0300000002036494
:0C036400787FE4F6D8FD7581240203AB1D
:1002CB00BC000BBE0029EF8DF084FFADF022E4CC17
:1002DB00F875F008EF2FFFEE33FEEC33FCEE9DECE0
:1002EB00984005FCEE9DFE0FD5F0E9E4CEFD22ED26
:1002FB00F8F5F0EE8420D21CFEADF075F008EF2F70
:10030B00FFED33FD4007985006D5F0F222C398FD60
:05031B000FD5F0EA22FD
:10032000C2D5EC30E709B2D5E4C39DFDE49CFCEEF8
:1003300030E715B2D5E4C39FFFE49EFE1202CBC3A3
:10034000E49DFDE49CFC80031202CB30D507C3E49E
:060350009FFFE49EFE2267
:0E035600C3E49FFFE49EFEE49DFDE49CFC22B8
:1003700002052EE493A3F8E493A34003F68001F270
:1003800008DFF48029E493A3F85407240CC8C3338E
:10039000C4540F4420C8834004F456800146F6DF5D
:1003A000E4800B010204081020408090055BE47E8D
:1003B000019360BCA3FF543F30E509541FFEE49352
:1003C000A360010ECF54C025E060A840B8E493A319
:1003D000FAE493A3F8E493A3C8C582C8CAC583CA44
:1003E000F0A3C8C582C8CAC583CADFE9DEE780BEFC
:010568000092
:00000001FF
